:030000000219FDE5
:03000B000200AA46
:03002B0002015D72
:03005B000202ECB2
:030073000202D9AD
:1000800002030406080C10182030406080040608A3
:100090000C10182030406080A0C00003070F1F0D17
:1000A0000D0403060D0503030202C2AFC0D0C0E079
:1000B000206214E5256009E473E525F4F58AD2622F
:1000C000D0E0D0D0D2AF3285268AC262E526F46075
:1000D0003030682620720DD0E0D0D0C290C287C2E6
:1000E00091D2AF32C290C287C291206F0D20660AB2
:1000F0007401D5E0FDE57BF45290D0E0D0D0D2AFD2
:1001000032758A00C28DD26201FA01B930680520C9
:100110006602D29001B9306805206602D28701B923
:10012000306805206602D29101B9D29630680A2063
:1001300066077405D5E0FDD29001B9D29430680A03
:100140002066077405D5E0FDD28701B9D2953068E5
:100150000A2066077405D5E0FDD29101B9C2AFC28D
:10016000AD53E6EFC0D0C0E0D2D3D2AFC2CEE52AC5
:100170006007207449152A21BE7800790020742E6A
:10018000E580307E01F430E60278FF53DACF207E3E
:100190000343DA20307E0343DA10C2D8C271E5800F
:1001A000307E01F430E60279FFC3E89970CB30610C
:1001B00003752A40207403752A40885CD27020742D
:1001C0000DE52B6004152B21CE43DA01C2D8207037
:1001D0000221E1A85C206102C27020740221DF8844
:1001E000227882B60403852224C3E5259440400288
:1001F000D26420CF0AD0E0D0D043E610D2AD32C2D4
:10020000CF053A7802E52A6005307402152AC3E565
:100210005C94014005755F00412B756000756900B5
:10022000E55F2401F55F5003755FFF7982B7020D2A
:10023000306E1DC3E52294324016854C227982B778
:10024000030E306E0BC3E52294324004798E872270
:10025000C3E5239522600840041523415F0523D898
:10026000CA0569E56970021569D56A63756A01781E
:1002700005C3E569956B4057C3E569956C500878EF
:1002800001756A03020293C3E569956D5005780113
:10029000756A01C3E5629524401E7982B704024164
:1002A000C4206E14852462E569046003856B69755A
:1002B0006A0175233C0202CFE5622850057562FF92
:1002C00041C4F562E5620470067560FF7569FFD090
:1002D000E0D0D043E610D2AD32C2AF53E67F759284
:1002E000FA7593FFC260759104D2AF32C2AF53E684
:1002F000EFC2ADC0D0C0E0C0F0D2D3D2AFA8FBA94E
:10030000FCC2D8307102615353DACF207E0343DA46
:1003100010307E0343DA20D271E580307E01F42074
:10032000E602612A88278928A13853DACF207E0384
:1003300043DA20307E0343DA10C2D8C2713074022F
:10034000A1247800E580307E01F430E602A1248803
:100350005CA10C53DACF207E0343DA20307E0343C6
:10036000DA10C271206102812C53DACF207E034360
:10037000DA10307E0343DA20C2D8D2718857895808
:10038000C3E89555F8E99556F97B007E087A00C3D5
:10039000E8948CE994005005755B00811E882178F3
:1003A000A2E6A8216055C3E894C8E994005008E487
:1003B000D2E4FB7A0A61F9C3E89468E99401500831
:1003C000E4D2E3FB7A0F61F9C3E894D0E9940250D8
:1003D00008E4D2E2FB7A1E61F9C3E894A0E994052F
:1003E0005008E4D2E1FB7A3C61F9C3E89498E994BF
:1003F000085008E4D2E0FB7A787E00C3E89559FC07
:10040000E9955AFD30E70AECF42401FCEDF43400E0
:10041000FD755B00C3EC9AED9E5003755B01885936
:10042000895A8557558558567802A10CC3E89527F7
:10043000F8E99528F9307C0281F0307B0281F030B8
:100440007A0281E9207502814FE9FDE8FC816EE9BD
:10045000C313F9E813F830790281E9E9C313F9E825
:1004600013F830780281E9E9C313FDE813FC206139
:0F0470002CC3EC941CED940240028185ED701EAC
:10047F00C3EC94C850180529E52970021529C3E566
:10048F0029940A5002A124755C00D270A124E52999
:10049F00600215297400207F037896E624FAFEE4A3
:1004AF003400FFC3EC9EFCED9FFD500678007900F1
:1004BF0081F0C3EC94FFED9400400678FF79008142
:1004CF00F0EC8572F0A4C5F0A2F733F87900400381
:1004DF0002050C78FF790002050CE9C313F9E81344
:1004EF00F8307C0EE9600278FFC3E81338F8E43483
:1004FF0000F9C3E894FFE99400400278FF885CD2CA
:10050F0070206102A124741FF4552F4BF52FC27474
:10051F00EB7002D274752A40307403752A0A306169
:10052F0002A13820740353DAFE207403752B20D0F8
:10053F00F0D0E0D0D0D2AD43E61032790102056899
:10054F007903020568790A020568791E0205687940
:10055F006402056879C80205687817E4D5E0FDD80C
:10056F00FAD9F6227A147B7802058F7A107B8C02E7
:10057F00058F7A0D7BB402058F7A0B7BC802058F2E
:10058F007902E4D294D5E0FDD287D5E0FDC287D5BC
:10059F00E0FDC294D5E0FDE920E002D29030E00208
:1005AF00D291E573D5E0FDE920E002C29030E00280
:1005BF00C2917496D5E0FDD9C9EAF8D5E0FDD8FB14
:1005CF00DBBED29422C37C007D0075F00005F0EAFB
:1005DF0033FAEB33FB50F6EB13FBEA13FAC3E9FFE5
:1005EF00E8FEE89AF8E99BF95004EFF9EEF8B3EC5E
:1005FF0033FCED33FDD5F0DFEDF9ECF822E889F0AF
:10060F008A20D2D4F8A9F07B0030F70B7BFFF424BB
:10061F0001F8E9F43400F9E88520F0A4ADF0F8E929
:10062F008520F0A4AFF0FEED2EF974003FFA7C04A4
:10063F00C3EA13FAE913F9E813F8DCF48BF030F797
:10064F000AE8F42401F8E9F43400F9E889F0C2D497
:10065F00F8A9F0227882B60403020702C3E55C947E
:10066F0019401EE52D54067018206E3678057994C2
:10067F00E7146007780A1460027812C3E5419840C6
:10068F001F306E098564627569FF756A01852224C2
:10069F00E4F544F545F546F547F548C26E02070205
:1006AF00D26E7994E7147013E523F43333F913F80A
:1006BF00E9540104F9E854FE0206F6E71414701425
:1006CF00E523F4333333F913F8E9540304F9E85409
:1006DF00FC0206FEE523F433333333F913F8E95400
:1006EF00070404F9E854F8C39440F8E99400F98832
:1006FF0044894522C3E54113F9E54013F8C3E544A6
:10070F0098F8E54599F9500CC3E89480E994FF40B7
:10071F001602073AC3E8947FE99400500302073AA0
:10072F00787F790002073A788079FF8849894A22D1
:10073F00E5492546F8E54A3547F9854A20E430076B
:10074F0001F43548FA30E709C3EA94F0401502077F
:10075F0078C3EA940F500302077878FF79FF7A0F76
:10076F00020778780079007AF0C3E5249561500A82
:10077F00C374019524500B020796E54A20E70E0239
:10078F000796E54A30E706884689478A482278A5C2
:10079F00E6FAC3E54933F8E54A33F9D10CE930E716
:1007AF000BC3E89480E994FF4013E1D0C3E8947F32
:1007BF00E994005002E1D0787F7900E1D078807918
:1007CF00FFE820E715C3E52398F84009C3E8940133
:1007DF0040030207F778010207F7E8F42401252305
:1007EF00F840030207F778FF884B2278A6E6FAA8AD
:1007FF0047A94812060CE930E70CC3E89401E994C5
:10080F00FF401602082CC3E894FFE994005003023E
:10081F00082C78FF790002082C780179FFE920E78E
:10082F0015C3E54B98F84009C3E89401400302084B
:10083F00537801020853E8F42401254BF8400302D2
:10084F00085378FF88242278FFC26420693D206A0C
:10085F0012D264C3E541940A4009C3E52594405080
:0E086F0002C26479A1E76023E541601F74FFB7
:10087D008541F0848539F0306A0375F005A4F8C51B
:10088D00F0600278FFC3E895645002A86488632283
:10089D00C3E5409440E5419401E56350031401AE76
:1008AD00046002F563227883E6F520120F2A75E8BD
:1008BD009012054A75E890E5E820ECFBA8BDA9BEAD
:1008CD00120FD0756E80756F02C3740213FD7480A4
:1008DD00606613FC74802CFC74023DFDECFAEDFB9C
:1008ED00C3E89AE99B4014E56E2480F56EE56F34FC
:1008FD0002F56FEA2CFAEB3DFB80E5AE6EAF6FC3F0
:10090D00E56F13F9E56E13F8C3E913F9E813F87AF7
:10091D0003C3E913F9E813F8DAF7AA201A70097579
:10092D006E00756F000209451AEA6008EE28FEEFA9
:10093D0039FFDAF88E6E8F6F2275E890227883E694
:10094D00FFE5E820ECF7A8BDA9BE0570C3E57094DE
:10095D00084052757000E9FA79A0E76044EA700723
:10096D00E571601B020980C3E895716010E5715057
:10097D0006600C1402098C0460F902098CE571F50E
:10098D0071C39467401B7561C0C3940440137561B6
:10099D0080C39404400B756140C39404400375619A
:1009AD000075BB0A22EFC39401601F7480601BC3E6
:1009BD00E894FFE994035012C3E8956EE9956F50E2
:1009CD0009E561600C15610209DEE561F46002055F
:1009DD0061A861C3E524985002A824C3E89562403C
:1009ED000AA862E562F4600385626188258826E5C0
:1009FD0070B4070375BB1022743279A787F0A4C5B4
:100A0D00F0A2F733F8C3E895614002A86188228807
:100A1D0024882588268864227540007541F022C2FD
:100A2D00AF75C820A8CCA9CDAA3A30CF010A75C898
:100A3D0024D2AFAB3BAC3C883B893CC3E89BF8E987
:100A4D009C206908F930670261384195AD3D8A3DBA
:100A5D00F9EA9DFA600478FF79FFAE3EAF3F8B3E19
:100A6D008C3FA83BA93CC3E89EF8E99FF9C3E5413B
:100A7D0013FBE54013FAE82AF540E93BF541500632
:100A8D007540FF7541FF41DFAA40AB41AC40AD4120
:100A9D007E047F02C3EB940440021E1FC3EB940837
:100AAD0040021E1FC3ED13FDEC13FCDEF7C3EA9CE1
:100ABD00FAEB9DFBEF6009C3E913F9E813F8DFF7D3
:100ACD00EA28FAEB39FB8A408B4150067BFF8B40BD
:100ADD008B41C3EB94025002D2673069047F0361EE
:100AED000A7892E6FFC3E537948240110FC3E537CC
:100AFD0094A040010FC3EF940640027F057E02E5EE
:100B0D0041C4540FF9E541C454F0F8E540C4540F05
:100B1D0028F8C3E89EFAE99400FB4009C3EA940261
:100B2D00EB940050047A02E4FB6184AA40AB41EBE4
:100B3D00C4FEEAC4540F4EFCC3EA9CFAEB9400FBCE
:100B4D00C3E813C313F8EA28FAEB3400FB8A408B91
:100B5D0041C3EB94024002C2677802EBC4FE7B00F6
:100B6D00EAC4540F4EFAC3EA98FA4005C3940250F2
:100B7D00027A027892E6FF30600261848551928597
:100B8D005293D26043E680C3E49AF8E49BF9306750
:100B9D00028110E8FAE9FBD3E913FDE813FC885153
:100BAD008952C3EF94036038EF20E00DE82CF8E98B
:100BBD003DF9ECFAEDFB020BD9E828F8E939F9C358
:100BCD00E82402F8E93400F97AFE7BFFC3EF9403C1
:100BDD00400E8A538B54884D894E8C4F8D508144D5
:100BED00885389548A4D8B4E8C4F8D5030691275B8
:100BFD0053F07554FF754FF07550FF7551F07552E8
:100C0D00FF8144E8FAD3E813FC8851C3EF940360E5
:100C1D0020EF20E007E82CF8ECFA8130E8282402D8
:100C2D00F87AFEC3EF940340088A53884D8C4F81A8
:100C3D004488538A4D8C4FE568C3335002646BF57D
:100C4D0068306002814E753402D26043E680E52D36
:100C5D0054066034A840A941C3E913F9E813F8C359
:0F0C6D00E913F9E813F8306904E92440F9C2AF3C
:100C7C0053E67F759100C3E498F594E499F5957566
:100C8C009104D26043E680D2AF22D26575430075E1
:100C9C002000306C03752040020CB5D26575430002
:100CAC00752040306C037520007801790120672095
:100CBC00E52D54066002C2657914E541C313700139
:100CCC0004F8C3941440027814306904781B791B1F
:100CDC00206010E543600C306903D53404D26DA15B
:100CEC005791560543E59B5440B52002A14130690C
:100CFC000908C3E89940011881DC20650A08C3E89B
:100D0C0099400281B581DCC265C2AF53E67F759113
:100D1C00003067127594007595FE759104D260438E
:100D2C00E680D2AF81B5AE40AF41C3E49EF594E40A
:100D3C009FF595A126C3E5339401500281B530652A
:100D4C000281B5D802A15581DCC26DC2AF53E67FDA
:100D5C00759100855394855495759104854D9285B4
:100D6C004E93D26043E680D2AFE52D540660082046
:100D7C006A020533020D93306D0D206C0A20650755
:100D8C001581158102160E2278003064053065023B
:100D9C007801E53775F007A4F9E5F028F5F0E9A23C
:100DAC00F013A2F113A2F213F537C3947850037524
:100DBC003778C3E53795384008D266C290C287C2EF
:100DCC0091306002A1CD854F92855093D26043E65D
:100DDC008022207D16C2AF754202D294C296306238
:100DEC0002D291D2AF759F34020FCDC2AF754202C1
:100DFC00D294C295306202D290D2AF759F34020F5A
:100E0C00CD307243207D20C2AF75420390013B75FB
:100E1C007B10C291D295306204D287C12BC294D27E
:100E2C00AF759F35020FCDC2AF75420390013B7574
:100E3C007B10C290D296306204D287C14BC294D23E
:100E4C00AF759F32020FCD207D17C2AF7542039054
:100E5C000116C291306202D287D2AF759F35020F54
:100E6C00CDC2AF754203900116C290306202D28798
:100E7C00D2AF759F32020FCD207D16C2AF754204E2
:100E8C00D296C295306202D287D2AF759F32020FD2
:100E9C00CDC2AF754204D295C296306202D287D2CF
:100EAC00AF759F35020FCD307243207D20C2AF75D8
:100EBC00420590012A757B40C287D294306204D2DD
:100ECC0090C1D1C296D2AF759F34020FCDC2AF750F
:100EDC00420590014C757B20C287D294306204D2BB
:100EEC0091C1F1C295D2AF759F34020FCD207D1701
:100EFC00C2AF75420590010CC287306202D290D20B
:100F0C00AF759F34020FCDC2AF754205900120C260
:100F1C00873062EBD291D2AF759F34020FCD207D1A
:100F2C0016C2AF754206D295C294306202D290D2EC
:100F3C00AF759F35020FCDC2AF754206D296C294E3
:100F4C00306202D291D2AF759F32020FCD30724314
:100F5C00207D20C2AF75420190014C757B20C29060
:100F6C00D296306204D291E177C295D2AF759F329E
:100F7C00020FCDC2AF75420190012A757B40C29120
:100F8C00D295306204D290E197C296D2AF759F355C
:100F9C00020FCD207D17C2AF754201900120C29087
:100FAC00306202D291D2AF759F32020FCDC2AF75B3
:100FBC00420190010CC291306202D290D2AF759F67
:100FCC0035C2662290010A757B00C290C287C2911D
:100FDC00D296D294D295C262227880760708760790
:100FEC000876010876040876FF0876FF08760B0869
:100FFC007602087601087601788C7601087600086E
:10100C0076B40876FF0876FF0876FF087603087634
:10101C00FF0876010876FF0876250876D0087678E2
:10102C000876C80876040876FF087601087600086A
:10103C00767A087607087601087601087600087635
:10104C00FF087600227887E6FFC272BF0302D272D5
:10105C007888C27DE630E102D27DC27E7889E630A6
:0F106C00E102D27EC3EF94026008758E01D27349
:10107B00021083758E00C273227880E61490008074
:10108B009378A5F67881E6149000809378A6F6788D
:10109B0086E61490008D9378A7F6789FE6F870019A
:1010AB0008C3E8941140027811E82828F56B256BEA
:1010BB00256B28F56C256B2828F56D7886E6F539B8
:1010CB00C394025003753902789CE67538FFB4025D
:1010DB00037538A0B4030375388278A3E614900027
:1010EB009A93F566120FD022227896E6FA7897E655
:1010FB00FB7888E6B40305C3EB940EFB307F047AD0
:10110B00007BFFC3EB9AFCC3948250027C82757206
:10111B00000572EC8572F0A4C3E5F0947D40F222D9
:10112B00D27F11F41205597A007B007C1012054F07
:10113B00E55C2AFA74003BFBDCF37C04C3EB13FB8A
:10114B00EA13FADCF7FEC27F11F422E5EF20E60387
:10115B007520000520903FFFE520146006901FFFCF
:10116B001460009304600375EF107597DE7597ADEF
:10117B007581C043FF8012054A75EF0075A900E524
:10118B00C7240220E70DF521E5B120E0068521C734
:10119B0043B101120FD07580FF75A48075F1C27534
:1011AB00D4BF75907475A57375F27B75D50475A650
:1011BB000175E34075E201120FD0E4F8F6D8FD7526
:1011CB006801120FE512166578988673753001C2A7
:1011DB00AF12056312057312055912057A120559E0
:1011EB001205811205591217881205631205631235
:1011FB00055EC2AF78FA79FA308607D9FBD8F702C9
:10120B001C001151118411F311F478988673120F8D
:10121B00D075881075890275C82475910475D840EE
:10122B0075A82275B80275E690759B80759D007543
:10123B00D1BC75BC5875BB0A75E88075B201120537
:10124B004AD2AF1208B375360053DACF207E034370
:10125B00DA20307E0343DA1043DA01C2D8C27112AE
:10126B000563D2617B037A0CE55B70077A0CDB03B9
:10127B000211FD1205592070030211FDC270E55CCD
:10128B00C3940240E1E52F541F855E5DF55EB55DAD
:10129B00D5DAD5C26153DACF207E0343DA20307E14
:1012AB000343DA10C2D8C27178A2E67008D274E593
:1012BB002F54E0F52FC27575290012055E307409A5
:1012CB00C3E529940A4002D27512054F7802307497
:1012DB00027800C3E55C9840F0C2AF1205731205AB
:1012EB0073120573D2AF120563754C0012054F785C
:1012FB008CE6C3940150030213CDE530C394015027
:10130B00030213CD207435C3E55C94FF5003021325
:10131B00CDC2AF120588D2AF12055EC3E55C940156
:10132B0050EFC2AF120573120554120573D2AF12F0
:10133B00055EC3E55C94FF40E902180D7F05D27F83
:10134B0011F412055EC2AFC27F11F4AE5CC3E55C53
:10135B00947FD2AF407612054AC2AF120588D2AF46
:10136B00DFDC312BC3EE94057897F612056312166A
:10137B00A71217907F0AD27F11F412055EC2AFC27B
:10138B007F11F4AE5CC3E55C947FD2AF50E61205DF
:10139B004AC2AF120573120554120573D2AFDFD6D2
:1013AB00312BEE24037896F61205631216A712174B
:1013BB00BF12055E11F4C3E55C94FF5002610F028E
:1013CB00180DC3E55C954C4003855C4C12055E78AB
:1013DB00017988E7B403027805C3E55C98400241C4
:1013EB00F7C2AF120588120588120588D2AF120515
:1013FB0063753000E4F531F5320531E531F4703FBA
:10140B000532789AE67819146012783214600D78E8
:10141B007D14600878FA146003753200C3E53298C6
:10142B00401D120FD012054A15327531007899867E
:10143B0073C2AF120588D2AF7898867312055E120D
:10144B000554E52A700530740221FD7801207402E1
:10145B007806C3E55C9840A112055EE52A7003028D
:0E146B0011FDC2AF120FD0E4F522F523F524D7
:10147900F525F526F567D2AF7885E6C333F565E43A
:10148900F544F545F546F547F548F570F52CF52D84
:10149900F53775700875BB1012054A120946E5E85B
:1014A90020ECFBA8BDA9BEE97001F8887112094AB0
:1014B90075700875BB101151C2AF7561FF120A052D
:1014C900852261852262852263D2AF752201752446
:1014D90001752501752601856069756A017888E6B7
:1014E900B40307C27D307602D27DD268D2697533E2
:1014F90000120F2A120F59120A25120A2C120A2554
:10150900120A2C120A25120CA7120663120D941244
:101519000DDE120A2C120C96306E03120703206797
:101529000312085630670312089D120D94120E0D0E
:10153900120A2C120CA7306E0312073F120D9412D7
:101549000E84120A2C120C96306E0312079D120D8E
:1015590094120EB3120A2C120CA7306E031207FA5A
:10156900120D94120F2A120A2C120946120C961205
:101579000D94120F5912094A120A2C30692C8564EC
:1015890061856462856069756A0179187A0CC3E5B9
:1015990033994009C269D26A8A350215B3C3E55C39
:1015A9009401400302150F021616306A1D206C1AA9
:1015B900E535147006C26AD26BA10FF535C3E55C37
:1015C9009401400302150F021616753600C3E55F34
:1015D90094014009856462856069756A0178FA79C0
:1015E900A4E760027803C3E55F985021307404E5ED
:1015F9002A601A78F0306C058564617820C3E5416A
:10160900985002A10F0536E55C6002C119753600D4
:10161900C2AF120FD07887E6FE760211517887EEB5
:10162900F6E4F522F523F524F525F526F565752C5F
:1016390000752D00D2AF12055E120FD078A4E660B6
:1016490006D290D287D291307406E52A700221FD24
:10165900788DE6C39401400241D461FF901A0D7858
:10166900201216E9E520B4A50CA31216E9E520B469
:101679005A03021687120FE51216A70216A6901A28
:101689000378807B0A1216E9A308DBF9901A0F7810
:101699008C7B191216E9A308DBF9901A2822C2AF2C
:1016A900121728121702901A00740E1216EEA3745C
:1016B900061216EEA374151216EE901A0378807BA3
:1016C9000A1216EDA308DBF9901A0F788C7B191210
:1016D90016EDA308DBF912173B121719901A2822E5
:1016E900E493F622E6438F01538FFD75EF0275B738
:1016F900A575B7F1F0538FFE22438F02438F017511
:10170900EF0275B7A575B7F1901A0DF0538FFC224A
:10171900901A0D74A5D1EE901A0E745AD1EE227A50
:101729003079D07820901A40D1E9E520F709A3DA79
:10173900F7227A3079D0901A40E7D1EE09A3DAF985
:1017490022AB74A875BB01027980BB02027981BB07
:1017590003027982BB04027994BB05027983BB0633
:10176900027986BB07027992BB08027987BB090215
:10177900799CBB0A027988BB0B027989E8F7227C3C
:1017890005120563DCFB22C2AF12057312057A123A
:10179900058112058812055412057312057A12057E
:1017A9008112058812055412057312057A120581F2
:1017B900120588D2AF22C2AF12058812058112051F
:1017C9007A12057312055412058812058112057AD9
:1017D90012057312055412058812058112057A1231
:1017E9000573D2AF22AE74AF75C2AF12057312057D
:1017F90073120573120554DEF2120588120554DFBF
:10180900F8D2AF221217901217881217887574012F
:101819007575017576001217EE7C05AD5C120563CE
:10182900C3ED955C70F5C3E55C9401400AC3E55CC2
:1018390094FF403702185112174A1216A71217902F
:10184900C2AF75EF10121788DCD10576C3E576941F
:1018590003500280C11217880575E5741490009F22
:0E18690093F808C3E57598500280A8121788FE
:101877001217880574C3E574940C50028094120FF4
:0C188700E51216A7C2AF75EF101217880B
:0319FD000211567E
:101A00000E061507070104FFFF0B020101A55A018D
:101A100000B4FFFFFF03FF01FF25D078C804FF01DA
:091A200000FF07010100FF00FFB7
:101A4000234638355F3341232020202020202020CA
:101A500023424C48454C492346383530232020202A
:101A60002020202020202020202020202020202076
:101C0000C2AFC2D37597DE7597AD7581C075A90057
:101C100043FF80752438752503B1C875EF0275E35D
:101C20004043F14053A4BF75D4FFD2867DFA7803B8
:101C300079E67C10752200752300901DD57B067512
:101C400024987525013086028145208608D8FBD965
:101C5000F9DCF781B7308608D8FBD9F9DCF781B712
:101C6000B188E493A3C39A6004DDC381B7DBDBB121
:101C70007A6002812E7B08E493FAA3B15BDBF87AE9
:101C800030B15B752200752300B17AEAFCEBFDC32D
:101C9000ED94FE400EB17A8A278B28ED30E0048A5D
:101CA000828B83B17A7AC270D8C3ED94FE601350F0
:101CB000CEBD0023EC60097520007521FF020000F5
:101CC0008100A827A9280809D804D90281D4B17EA7
:101CD000EAF281C80D81A3C3ED94035047EDA2E061
:101CE00092007AC5C3E5829400E583941C5092204B
:101CF0000010438F02438F0175B7A575B7F1F0301F
:101D0000001DA827A9280809438F01538FFDD80477
:101D1000D902A11FE275B7A575B7F1F0A3A10E53C3
:101D20008FFC817F7AC1BD030CE493A3FAB13FDC41
:101D3000F8B137817F8181AA22AB23B15BEBFAEA4C
:101D40006222752608C3E52313F523E52213F52245
:101D500050066323A0632201D526EAB1C8B1C87535
:101D6000260AEAF4200102D286300102C286B1C8F6
:101D7000C3134002C201D526EB22B17EEAFB2086C6
:101D800002A17E308602A183752608AE24AF25C34A
:101D9000EF13FFEE13FEB1CCB1C8C3EA13308602D5
:101DA0004480FA30E703632201C3E52313F523E5FA
:101DB0002213F52250066323A0632201D526D9E51C
:101DC0002265236523F52222AE24AF250E0FDEFE09
:101DD000DFFCD20122424C48656C6934373163F82C
:031DE000500601A9
:00000001FF
